:020000040000FA
:020000000528D1
:0800080005288316FF23900078
:100010000830850000308100083096008312850189
:100020000730990008308B000630A80066209A201F
:10003000850190206620692090208501902066200F
:10004000692090208501902066206920851D262842
:1000500096201E30A5006430A6009B30A7000C300F
:10006000A400851D4328A40B3128A70B2F28A60B1D
:100070002D28A50B2B2869209320692085010B10C2
:100080006300000016280630A4072408A9005520A4
:100090008A2085194C28472855209620851D4528FB
:1000A000A90B4C289D207220262828085E20850058
:1000B0006920A80B08000630A800080082071F343A
:1000C00009340A340B340E340F341E3417308500D3
:1000D00008003030A00085167C2085127C20A00B03
:1000E0006B280800692093206920932069209320C1
:1000F00069209320692008003030A100A10B7E28E0
:1001000008000830A2007D30A300A30B8528A20BB5
:1001100083280800812081208120812081200800FF
:100120008A208A20080090209020080090209320A8
:10013000932008009620962008009A209A209A2062
:020140000800B5
:0207FE00D834ED
:02400E0084111B
:00000001FF
